:10000000F9C0000015C1000013C1000011C10000BB
:100010000FC100000DC100000BC1000009C10000AC
:1000200007C1000039C7000036C4000001C100004C
:10003000FFC00000FDC00000FBC00000F9C00000D0
:10004000F7C00000F5C00000F3C00000F1C00000E0
:10005000EFC00000EDC00000EBC00000E9C00000F0
:10006000E7C00000E5C00000E3C00000E1C0000000
:10007000DFC00000DDC00000DBC00000D9C0000010
:10008000D7C00000D5C00000D3C00000D1C0000020
:10009000CFC00000CDC00000CBC00000C9C0000030
:1000A000C7C00000C5C00000C3C0000012010002AC
:1000B00000000040000000000010010200010902E1
:1000C0003B00020100C032090400000103000200ED
:1000D00009211101000122340007058103080006EF
:1000E000090401000103000101092111010001229D
:1000F0003B00070582030800140C034F0054004C1A
:10010000004C0043002603430068006F0072006447
:10011000006900740065002000500072006F0074D8
:10012000006F007400790070006500040309040585
:10013000010902A1010901A10005091901290315FD
:100140000025017501950381027505950181010561
:10015000010930093109381581257F75089503811A
:1001600006C0C005010906A101050719E029E71528
:100170000025017501950881028101190029651585
:1001800000256575089506810005081901290515E2
:1001900000250175019505910295039101C0002C80
:1001A0002AE1080C11061712160915101A14040B6F
:1001B000071C0F13050D180A191B0E1D002B3637CF
:1001C00033342F3031381E1F2021222324252627A7
:1001D0002D2E2835E2E0504F52514B4E494C4A4D9E
:1001E0004648E539E3E73A3B3C3D3E3F4041424328
:1001F0004445292911241FBECFEFDAE0DEBFCDBF71
:1002000081E011E0A0E0B1E0E4E9F3E102C0059093
:100210000D92A430B107D9F711E0A4E0B1E001C01C
:100220001D92AC32B107E1F70E94C1090C94C809D4
:10023000E7CE8FB7F89497EF94BF98E10FB6F89494
:1002400090936000109260000FBE87FF01C0789409
:100250000895F2D3E5D60E947C09FBCFEFD309D6EF
:10026000E1C7FCDFF6CF13BE83B7856083BF8895F7
:1002700008959091EB0091609093EB008093EC00D7
:100280008091ED008270862B8093ED008091ED00CF
:1002900082608093ED008091EE00881F8827881F80
:1002A00008951092E9008091EB0080FF02C080E089
:1002B00008951092E9008091EB0081608093EB003B
:1002C00082E08093EC008091ED00827080638093E7
:1002D000ED008091ED0082608093ED008091EE0052
:1002E000881F8827881F08957894E8EDF0E08081C2
:1002F0008F7680838081806980837894089582E1FD
:1003000089BD09B400FEFDCF8091D8008F7D809318
:10031000D800C7DF8091E0008E7F8093E00080915D
:10032000E20081608093E2008091E2008860809327
:10033000E20008958091D90080FF14C080910401EB
:10034000882381F481E0809304011092060191D505
:100350008091080190910901826090930901809336
:100360000801CDDF8091D90080FD13C02FC010920D
:10037000040110921E01809108019091090184608E
:1003800090930901809308018091D8008062809346
:10039000D800809108019091090190FF10C08091D0
:1003A0000801909109019E7F9093090180930801B3
:1003B00081E08093EA001092EA0010921E011092F0
:1003C000E9008091E80083FF06C01FC0809104010E
:1003D0008130F9F6CCCF089509B400FC05C082E164
:1003E00089BD09B400FEFDCF8091D8008F7D809338
:1003F000D80080910601813039F48091E00082605C
:100400008093E0001092060108950F931F93DF93ED
:10041000CF9300D0CDB7DEB78091E8008B7F80937B
:10042000E8001091F1000091F1000630F9F007307A
:1004300068F4013009F413C1013008F498C10330A5
:1004400009F44FC1053009F00DC2D2C0093009F4DA
:10045000EFC00A3020F4083009F004C2A4C00A300A
:1004600009F4BBC10B3009F0FDC1DAC1103809F045
:10047000F9C16091F1008091F100813019F0823072
:1004800089F406C082E180931F018CEA90E005C0E8
:100490008BE380931F018EEB90E09093210180937A
:1004A000200104C0E8D2882309F4DCC18091F10066
:1004B0008091F1008091F10089838091F1008A831D
:1004C0008091E800877F8093E80029813A818091BC
:1004D0001F0190E08217930730F48F739070892B7F
:1004E00021F461E003C020931F0160E08091E800E7
:1004F0008F7E8093E800209120013091210140916E
:100500001F0122C08091E80084FF03C0F90190E040
:100510000FC08091E80080FFF5CFF8CF542F5150E5
:10052000903449F09F5F84918093F1003196452F7C
:100530009F01442399F78091E80084FD12C08091C7
:10054000E8008E7F8093E800442339F42093200153
:100550003093210110921F010AC08091E80084FFAE
:10056000D8CF209320013093210140931F016130A7
:1005700069F48091E80084FD09C08091E80080FF63
:10058000FCCF8091E8008E7F8093E8008091E800A6
:1005900084FFFCCF8091E8008F7E8093E8008091FB
:1005A000E8008B7F22C0103809F05CC18091E80020
:1005B000877F8093E80080911E018093F1008091F5
:1005C000E8008E7F8093E8008091E8008F77809329
:1005D000E8008091E80082FFFCCF8091E8008B7FEB
:1005E0008093E8008091E8008F778093E8004CC109
:1005F000112309F037C19091F1008091E3009F77BA
:100600008078982B9093E3008091E800877F809317
:10061000E8008091E8008E7F8093E8008091E800F8
:1006200080FFFCCF8091E30080688093E3002CC1C1
:10063000112309F017C19091F100923008F012C116
:100640008091E800877F8093E80090931E0180915D
:10065000E8008E7F8093E800892FF8D315C111231D
:1006600021F0123009F0FEC00DC08091F100813000
:1006700009F0F8C0809107018D7F809307011092E7
:1006800006016CC08091F1009091F100882309F07F
:10069000E9C0E091F100EF77E093E9008091EB0091
:1006A00080FF4DC0EE23B1F08091EB00806180931C
:1006B000EB0081E090E00E2E02C0880F991F0A9493
:1006C000E2F78093EA001092EA008091EB008860E4
:1006D0008093EB001092E900F0E0E95EFE4F10829B
:1006E0003DC0112321F0123009F0BCC00DC0909123
:1006F000F100913009F0B6C08091070182608093CB
:100700000701909306012AC08091F1009091F100B9
:10071000882309F0A7C0E091F100EF7751F48091B0
:10072000EB0080628093EB008091E800877F8093EC
:10073000E800E093E9008091EB0080FD03C0109297
:10074000E90090C08091EB0080628093EB001092F2
:10075000E900F0E0E95EFE4F81E080838091E800EF
:10076000877F8093E8008091E8008E7F3ECF809164
:10077000F1008091F100E091F100113869F0123838
:1007800099F0103809F06EC08091E800877F80935F
:10079000E8008091070113C08091E800877F809373
:1007A000E8001092F1000DC08091E800877F8093EF
:1007B000E800F0E0EF77F070E95EFE4F8081809313
:1007C000F1001092F1008091E8008E7F8093E800A4
:1007D0008091E80082FFFCCF00CF113809F042C0C1
:1007E0008091F1008091F1009091F10099839091B6
:1007F000F1009A838823B1F58091E800877F809388
:10080000E80089819A8120D18093F1008091E800ED
:100810008E7F8093E8008091E80082FFFCCFDDCEE0
:10082000113001F56091F1008091F1009091F1009B
:1008300099839091F1009A838823A1F48091E80034
:10084000877F8093E80089819A8100D11092E90026
:100850008091E8008E7F8093E8008091E80080FF1F
:10086000FCCF12C0812F602FABD2882369F4809116
:10087000EB0080628093EB008091E800877F80939B
:10088000E80081E0809317010F900F90CF91DF91E6
:100890001F910F9108951F920F920FB60F9211247E
:1008A0002F933F934F935F936F937F938F939F9378
:1008B000AF93BF93EF93FF938091E10082FF08C055
:1008C0008091E20082FF04C08BEF8093E100DED2D2
:1008D0008091E10080FF41C08091E20080FF3DC037
:1008E000809106018130D9F480911E018823B9F0EE
:1008F0008091E2008E7F8093E2008FEE8093E10092
:100900008091E20080618093E20089B58D7F89BD8E
:1009100019BC8091D80080628093D8001DC08FEEF2
:100920008093E10080910801909109018062909389
:100930000901809308018EEF8093E1008091E2002D
:1009400080618093E2008091D80080628093D8001B
:1009500089B58D7F89BD19BCCDD28091E10084FF1E
:1009600027C08091E20084FF23C009B400FC05C0C9
:1009700082E189BD09B400FEFDCF8091D8008F7D52
:100980008093D8008FEE8093E1008091E2008F7E0B
:100990008093E20080910801909109018064909316
:1009A0000901809308018091E20081608093E20058
:1009B0008091E10085FF1AC08091E20085FF16C09A
:1009C0008091E2008F7E8093E2008FED8093E100C2
:1009D0008091E2008F7D8093E200809108019091E8
:1009E0000901806890930901809308018091E100DA
:1009F00083FF11C08091E20083FF0DC087EF8093D9
:100A0000E1004FDC80910801909109019160909381
:100A1000090180930801FF91EF91BF91AF919F91E0
:100A20008F917F916F915F914F913F912F910F9097
:100A30000FBE0F901F9018957DCC0895E7EDF0E064
:100A400080818160808350CC80E00895892B91F46F
:100A500081E08093E9008091EB0080618093EB005E
:100A600082E08093EA001092EA008091EB008860B7
:100A70008093EB0008958330F1F4613059F06130D8
:100A800018F06230C1F40CC084E080931F018BE247
:100A900091E00BC08CE080931F0189EF90E005C0CE
:100AA00086E280931F0185E091E09093210180937D
:100AB000200181E0089580E00895DF93CF9300D076
:100AC00000D0CDB7DEB78091F1008B838091F1002B
:100AD0008C838B819C81009719F0019781F406C06B
:100AE00084E380931F018FE291E005C08BE3809344
:100AF0001F0183E691E09093210180932001809172
:100B0000F10089838091F1008A838091E800877FDA
:100B10008093E80029813A8180911F0190E082173B
:100B2000930770F48F739070892B11F461E001C00A
:100B300060E0209120013091210140911F011CC0F3
:100B400020931F01F5CF8091E80080FFFCCFF901D1
:100B500090E00AC0542F5150903449F09F5F849127
:100B60008093F1003196452F9F01442399F780919E
:100B7000E8008E7F8093E800442359F08091E800DC
:100B800082FFE1CF209320013093210140931F0188
:100B900006C0209320013093210110921F01809103
:100BA000E80082FD0FC0613049F48091E80080FFC9
:100BB000FCCF8091E8008E7F8093E8008091E80070
:100BC00082FFFCCF8091E8008B7F8093E8008091CA
:100BD000E8008F778093E8000F900F900F900F90B0
:100BE000CF91DF9108958091E800877F8093E8009E
:100BF0008091E8008E7F8093E8008091E80082FF7A
:100C0000FCCF8091E8008B7F8093E8008091E80022
:100C10008F778093E8008091E8008E7F8093E800D2
:100C20000895DF93CF9300D000D0CDB7DEB7809189
:100C3000F1008B838091F1008C838091F100898396
:100C40008091F1008A838091E800877F8093E8009B
:100C500089819A81892B49F080910A018093F10062
:100C60008091E8008E7F8093E8008091E80082FF09
:100C7000FCCF8091E8008B7F8093E8008091E800B2
:100C80008F778093E8000F900F900F900F90CF9187
:100C9000DF910895DF93CF9300D000D0CDB7DEB7BA
:100CA0008091F1008B838091F1008C838B819C81FA
:100CB000009719F0019781F406C089E080931F0125
:100CC00080ED90E005C089E080931F0189EE90E0FF
:100CD00090932101809320018091F100898380917C
:100CE000F1008A838091E800877F8093E800298162
:100CF0003A8180911F0190E08217930770F48F73FF
:100D00009070892B11F461E001C060E02091200116
:100D10003091210140911F011CC020931F01F5CF8C
:100D20008091E80080FFFCCFF90190E00AC0542FC9
:100D30005150903449F09F5F84918093F100319637
:100D4000452F9F01442399F78091E8008E7F80937F
:100D5000E800442359F08091E80082FFE1CF20931E
:100D600020013093210140931F0106C020932001F0
:100D70003093210110921F018091E80082FD0FC085
:100D8000613049F48091E80080FFFCCF8091E80059
:100D90008E7F8093E8008091E80082FFFCCF8091F5
:100DA000E8008B7F8093E8008091E8008F77809344
:100DB000E8000F900F900F900F90CF91DF91089562
:100DC000DF93CF9300D0CDB7DEB72091F1009091A3
:100DD000F100813859F4663099F5913219F0923268
:100DE00079F502C057DF2AC068DE28C0813201F5DC
:100DF000693019F06A3021F504C0923009F5F3DE4C
:100E00001DC08091F10089838091F1008A838091D7
:100E1000E800877F8093E80090930A018091E800C2
:100E20008E7F8093E8008091E80080FFFCCF06C0B1
:100E3000813A31F4623021F4822FF3DE81E001C087
:100E400080E00F900F90CF91DF9108950F931F9343
:100E500009EE10E081E0F801808381EC60E009DABE
:100E600082E0F801808381EC60E003DA1F910F914A
:100E7000089510922201E2EEF0E080818460808388
:100E80001092240181E08093230108958091220132
:100E90008F5F8093220108951F920F920FB60F92D9
:100EA00011242F933F934F935F936F937F938F936F
:100EB0009F93AF93BF93EF93FF93E8E6F0E08081B9
:100EC0008E7F8083D89AEBE6F0E080818F718083FB
:100ED00083DAFF91EF91BF91AF919F918F917F91B5
:100EE0006F915F914F913F912F910F900FBE0F9097
:100EF0001F90189580910601813059F480916B0004
:100F0000806E80936B00D89A809168008160809396
:100F100068007894A8C910922601109227011092B7
:100F2000280110922901F0D0482F882329F48091BC
:100F30000E01882321F472C08E3109F46FC0642F32
:100F400070E09B012F7030702A30310531F48091B0
:100F5000280181508093280125C02230310559F4A1
:100F600080912801815080932801809127018F5F13
:100F70008093270120C02330310531F4809127016F
:100F80008F5F809327011EC02130310559F4809175
:100F900028018F5F80932801809127018F5F8093C4
:100FA000270113C02530310531F4809128018F5F6E
:100FB0008093280117C02430310521F48091280145
:100FC0008F5F09C02C30310541F02830310551F4D4
:100FD00080912801815080932801809127018150C0
:100FE00080932701CB01807390708031910521F4AB
:100FF0008091260181600CC08032910521F480919E
:101000002601826005C0C09729F480912601846082
:101010008093260140930E0181E0089580E00895B9
:1010200080910F01882309F46EC080910B0190918B
:101030000C01019690930C0180930B01019794FF92
:101040004E9A8091D90080FF58C080911E0188235C
:1010500009F459C080912201833008F454C01092E1
:10106000220180912401882331F455DF882319F06F
:1010700081E08093240190912401992329F48091A7
:101080002301882309F43FC021E02093E9008091E7
:10109000E80085FF38C0992359F01092240110927E
:1010A000230180912601882369F0209323010AC03F
:1010B0001092260110922701109228011092290106
:1010C00010922301809126018093F10080912701E5
:1010D0008093F100809128018093F1008091290193
:1010E0008093F1008091E8008E7F8093E8008091EA
:1010F000E8008F778093E800089513BE83B785607A
:1011000083BF8895A2CF0895DF93CF9300D000D0FE
:10111000CDB7DEB783B18095898383B180958A830B
:1011200083B180958B8383B180958C8320E0BE0151
:101130006F5F7F4F09C083B1922F9370FB01E90F5E
:10114000F11D809580832F5F49818A81481799F727
:101150008B81481781F78C81481769F740931601F6
:10116000442329F4809115018823F9F452C04E31AB
:10117000E1F4809115018E31C1F080910F01882337
:1011800059F481E080930F0184E690E0909301018F
:10119000809300015E9A09C010920F0182E390E0F3
:1011A00090930101809300015E9890911501842F26
:1011B0008923891769F0109214011092130140934A
:1011C000150180910201882381F01092020122C052
:1011D000892F842B891759F081E0809302011092A6
:1011E0001401109213014093150190E013C0209157
:1011F0001301309114018091000190910101281791
:10120000390738F42F5F3F4F3093140120931301B7
:10121000ECCF942F892F0F900F900F900F90CF91BC
:10122000DF91089514B88FEF85B9569A1092250171
:10123000E2EEF0E08081846080830895982F882317
:1012400061F480911101803EE8F58823D9F1109274
:1012500011011092120120E04DC0833EF1F0843E56
:1012600038F4813E91F0823EA0F4803E59F509C0E9
:10127000853ED9F0853EA8F0863ED9F0873E11F52F
:101280001CC08091120181601BC08091120182609C
:1012900017C080911201846013C080911201886090
:1012A0000FC08091120180610BC080911201806299
:1012B00007C080911201806403C080911201806890
:1012C0008093120120911201222321F480911001B8
:1012D000882311F05E9A01C05E98993349F4809199
:1012E0001101893329F080911001809580931001BC
:1012F00090931101822F089580910F01882309F0A6
:101300003FC082E08093E9008091E80080FF38C010
:1013100080911E018823A1F18091E80080FFFCCF1D
:10132000F3DE80932B01863510F010922B01E091B3
:101330002B01F0E0E256FE4FE491E0932B0182E0B6
:101340008093E9008E2F7ADF8093F1001092F100F4
:1013500080912B018093F1001092F1001092F10026
:101360001092F1001092F1001092F1008091E800CB
:101370008E7F8093E8008091E8008F778093E8006B
:1013800008950E9419010E94310180E090E00895C3
:04139000F894FFCFFF
:041394003200010022
:00000001FF
